:020000040800F2
:1000000000C00020F9020008D5150008D915000825
:10001000DD150008E1150008E515000800000000E6
:10002000000000000000000000000000E9150008CA
:10003000ED15000800000000F1150008F515000896
:1000400065130008651300086513000865130008B0
:1000500065130008651300086513000865130008A0
:100060006513000865130008651300086513000890
:100070006513000865130008651300086513000880
:100080006513000865130008651300086513000870
:100090006513000865130008651300086513000860
:1000A0006513000865130008651300086513000850
:1000B0006513000865130008651300086513000840
:1000C0006513000865130008651300086513000830
:1000D0006513000865130008651300086513000820
:1000E0006513000865130008651300086513000810
:1000F0006513000865130008651300086513000800
:1001000065130008651300086513000865130008EF
:1001100065130008651300086513000865130008DF
:1001200065130008651300086513000865130008CF
:1001300000000000000000000000000000000000BF
:1001400000000000000000000000000000000000AF
:10015000000000000000000000000000000000009F
:10016000000000000000000000000000000000008F
:10017000000000000000000000000000000000007F
:10018000000000000000000000000000000000006F
:10019000000000000000000000000000000000005F
:1001A000000000000000000000000000000000004F
:1001B000000000000000000000000000000000003F
:1001C000000000000000000000000000000000002F
:1001D000000000000000000000000000000000001F
:1001E0005FF8E0F100B583B001F0ACF8304B314A74
:1001F0001360314A1360314B314A03E011681960D2
:10020000043304322F498B42F8D32A4B1A682E4B01
:100210009A4204D1284B1A682C4B9A4200D0FEE730
:10022000234B2B4A13602B4A13602B4B02E0002216
:100230001A600433294A9342F9D3254B1B6813B93A
:10024000244B1B6803B1FEE701F088F8694601A85A
:1002500001F070F8224C234B1C1BA410002504E075
:100260001F4B53F8253098470135AC42F8DC1E4C43
:100270001E4B1C1BA410002504E01B4B53F825301B
:1002800098470135AC42F8DC0099019801F04AF931
:100290000546174C174B1C1BA41004E0013C144BE3
:1002A00053F824309847002CF8DC284601F040F839
:1002B000BABADECA000000201000002000000020B2
:1002C0001C18000814000020785634123254769816
:1002D00014000020600100201400002064010020B0
:1002E0009403000894030008940300089403000892
:1002F000940300089403000808B5FFF773FF00BFDC
:1003000000BEFEE71EF0040F0CBFEFF30880EFF312
:1003100009807146124A104700BEFEE700BEFEE7A4
:100320001EF0040F0CBFEFF30880EFF30980714655
:100330000C4A104700BEFEE71EF0040F0CBFEFF39F
:100340000880EFF309807146074A104700BEFEE7B8
:1003500000BEFEE700BEFEE700BEFEE770470000FD
:0C03600019030008350300084D030008D5
:10036C001C18000800000020140000201C180008B5
:10037C0000000000000000001400002064010020B8
:08038C00000000000000000069
:1003940010B5044600F0C4FF064BA3FB00308009EF
:1003A40000F098F8002221464FF0FF3000F050F89A
:1003B400002010BDD34D621008B5074A136843F0FE
:1003C40010031360032000F025F80020FFF7E0FF7E
:1003D40001F0B6F8002008BD00200240024A13686C
:1003E40001331360704700BF18000020014B1868E8
:1003F400704700BF1800002010B582B00190FFF7CD
:10040400F5FF0446FFF7F2FF001B019B9842F9D366
:1004140002B010BD10B50446C31E042B03D9BA2183
:10042400094801F08BF8094AD36823F4E0631B04FC
:100434001B0C240204F4E064234343F0BF6343F43D
:100444000033D36010BD00BF6C17000800ED00E05E
:1004540070B504460E4615460F2A03D9D2211A4810
:1004640001F06CF80F2E03D9D321174801F066F878
:10047400164BDA68C2F30222C2F10701042928BF2D
:100484000421131D062B01D9033A00E000220123A5
:1004940003FA01F101393140914003FA02F2013AC1
:1004A4002A400A43002C06DA04F00F041201D2B2E7
:1004B400074B1A5570BD1201D2B204F1604404F521
:1004C400614484F8002370BD6C17000800ED00E05F
:1004D40014ED00E00138B0F1807F0AD2064B586079
:1004E400F021064A82F823100020986007221A603F
:1004F40070470120704700BF10E000E000ED00E00D
:1005040010B50446042805D020B14FF4DF71084823
:1005140001F014F8042C05D1064A136843F00403CF
:10052400136010BD034A136823F00403136010BD65
:100534006C17000810E000E008B501F07DF808BD74
:100544002DE9F04383B080460F46B54B98421BD04B
:1005540003F58063984217D003F58063984213D063
:1005640003F5806398420FD003F5806398420BD063
:1005740003F58063984207D003F58063984203D063
:10058400CF21A84800F0DAFF3B881BB9D021A54849
:1005940000F0D4FF7B68012B22D9112B20D0022B31
:1005A4001ED0122B1CD0A04A934219D002F58012FF
:1005B400934215D002F58012934211D0A2F5F8129D
:1005C40093420DD002F58012934209D002F58012B5
:1005D400934205D0032B03D0D121924800F0AEFF03
:1005E4004FF000094E463FE10125B5403C682C40E0
:1005F400A54240F038818A4B98451BD003F58063AF
:10060400984517D003F58063984513D003F58063AC
:1006140098450FD003F5806398450BD003F58063AC
:10062400984507D003F58063984503D0DF217D48C2
:1006340000F084FF7B68122B49D00CD8022B3AD0EF
:1006440004D8002B4FD0012B1ED067E0032B60D0C1
:10065400112B24D062E0754A934244D008D8A2F505
:10066400801293423FD002F58032934256D13AE051
:100674006F4A934237D002F58032934233D0A2F5C9
:10068400801293424AD12EE0FB68013B022B03D92E
:10069400E721644800F052FFD7F80C903EE0FB6875
:1006A400013B022B03D9EE215E4800F047FFFB68B3
:1006B40003F1040932E0FB68013B022B03D9F52165
:1006C400584800F03BFFFB6803F1080926E0FB688B
:1006D400013B022B03D9FC21524800F02FFFFB6899
:1006E40003F10C091AE0BB68022B04D940F209118A
:1006F4004C4800F023FFBB6873B1012B04D1C8F848
:1007040010504FF0080909E0C8F814504FF00809D8
:1007140004E04FF0000901E04FF00409FF2C01D878
:10072400404601E008F10400FF2C01D8B30002E0C8
:10073400A6F108039B0001680F229A4021EA0202F5
:1007440009FA03F3134303607B6813F0805F00F03E
:100754008A80384B9A6942F001029A619B6903F0DE
:1007640001030193019BB1088A1C334B53F8220007
:1007740006F003039B000F229A4020EA0200284A55
:10078400904515D002F58062904513D002F5806241
:10079400904511D002F5806290450FD002F5806239
:1007A40090450DD002F5806290450BD105220AE0F8
:1007B400002208E0012206E0022204E0032202E013
:1007C400042200E0062202FA03F3034302311A4A28
:1007D40042F821307B6813F4803F05D002F5806233
:1007E40013682343136004E0144A136823EA0403E0
:1007F40013607B6813F4003F04D0104A536823430A
:10080400536004E00D4A536823EA040353607B6891
:1008140013F4801F14D0094A93682343936014E0AF
:10082400000801409C17000800001110000021106E
:10083400000031100010024000000140000401409B
:100844000C4A936823EA040393607B6813F4001F43
:1008540004D0084AD3681C43D46004E0054AD36832
:1008640023EA0404D46001360F2E7FF6BDAE03B034
:10087400BDE8F0830004014070B5064615460C46F9
:1008840021B94FF4F271084800F058FE012D04D943
:1008940040F2E511044800F051FE0DB1346170BD21
:1008A4002404346170BD00BF9C17000838B50446A9
:1008B4000D4621B94FF4FD71034800F03FFEE16895
:1008C4006940E16038BD00BF9C17000830B583B0B3
:1008D400044620B94FF48771B94800F02FFE23680D
:1008E4003BB113F00F0F04D140F20F11B44800F0E4
:1008F40025FE236813F0010F00F0A380636853B151
:10090400B3F5803F07D0B3F5A02F04D040F2151102
:10091400AB4800F013FEAB4B5B6803F00C03042BF5
:100924000AD0A84B5B6803F00C03082B1BD1A54B22
:100934005B6813F4803F16D04FF4003393FAA3F3AB
:10094400A04B1A684FF4003393FAA3F3B3FA83F37A
:1009540003F01F0322FA03F313F0010F71D063684D
:10096400002B6ED11BE36368B3F5803F05D1954A34
:10097400136843F48033136026E063B903F18043C2
:1009840003F504331A6822F480321A601A6822F4D8
:1009940080221A6018E0B3F5A02F0CD103F1804334
:1009A400A3F53C331A6842F480221A601A6842F4B0
:1009B40080321A6008E0834B1A6822F480321A608D
:1009C4001A6822F480221A606368EBB1FFF70EFD07
:1009D400054605E0FFF70AFD401B642800F2E182AA
:1009E4004FF4003393FAA3F3764B1A684FF40033B1
:1009F40093FAA3F3B3FA83F303F01F0322FA03F386
:100A040013F0010FE6D01CE0FFF7F0FC054605E00B
:100A1400FFF7ECFC401B642800F2C5824FF400335E
:100A240093FAA3F3674B1A684FF4003393FAA3F3D2
:100A3400B3FA83F303F01F0322FA03F313F0010F55
:100A4400E6D1236813F0020F00F0A0802369012B84
:100A540004D940F249115A4800F070FD63691F2B14
:100A640004D94FF4A571564800F068FD554B5B68F6
:100A740013F00C0F0AD0534B5B6803F00C03082BE4
:100A840027D1504B5B6813F4803F22D1022393FAA1
:100A9400A3F34C4B1A68022393FAA3F3B3FA83F338
:100AA40003F01F0322FA03F313F0010F03D02369A9
:100AB400012B40F07A824348036823F0F80163690C
:100AC400F82292FAA2F2B2FA82F293400B43036044
:100AD4005CE023699BB3012292FAA2F3B3FA83F395
:100AE4009B0003F1844303F584031A60FFF77EFC43
:100AF400054605E0FFF77AFC401B022800F2578206
:100B0400022393FAA3F32F4B1A68022393FAA3F355
:100B1400B3FA83F303F01F0322FA03F313F0010F74
:100B2400E8D02848036823F0F8016369F82292FAB0
:100B3400A2F2B2FA82F293400B43036026E001234F
:100B440093FAA3F3B3FA83F39B0003F1844303F50D
:100B5400840300221A60FFF749FC054605E0FFF70D
:100B640045FC401B022800F22482022393FAA3F3DB
:100B7400144B1A68022393FAA3F3B3FA83F303F032
:100B84001F0322FA03F313F0010FE8D1236813F0D3
:100B9400080F5CD0A369012B04D94FF4C571084830
:100BA40000F0CCFCA3696BB3012292FAA2F3B3FA6E
:100BB40083F3054941F82320FFF718FC05460BE0B1
:100BC400E01700080010024080044242FFF70EFCC8
:100BD400401B022800F2EF81022393FAA3F293FA56
:100BE400A3F2A44A526A93FAA3F3B3FA83F303F089
:100BF4001F0322FA03F313F0010FE7D00120FFF7DC
:100C0400FBFB24E0012393FAA3F3B3FA83F300215B
:100C1400994A42F82310FFF7E9FB054605E0FFF780
:100C2400E5FB401B022800F2C881022393FAA3F2D9
:100C340093FAA3F28F4A526A93FAA3F3B3FA83F3B3
:100C440003F01F0322FA03F313F0010FE7D1236823
:100C540013F0040F00F0AB80E368012B06D9052BD9
:100C640004D040F2B711854800F068FC814BDA6982
:100C740042F08052DA61DB6903F080530193019BF7
:100C84007F4A136843F480731360FFF7AFFB054694
:100C940005E0FFF7ABFB401B642800F29081784B22
:100CA4001B6813F4807FF4D0E368012B05D1714AEB
:100CB400136A43F00103136222E063B903F1804332
:100CC40003F504331A6A22F001021A621A6A22F046
:100CD40004021A6214E0052B09D1664B1A6A42F029
:100CE40004021A621A6A42F001021A6208E0614BB5
:100CF4001A6A22F001021A621A6A22F004021A62C3
:100D0400E36853B3FFF772FB054607E0FFF76EFB9A
:100D1400401B41F28833984200F25381022393FA34
:100D2400A3F293FAA3F3B3FA83F35B0943F0020348
:100D3400DBB2022B02D14F4B1A6A01E04D4B5A6AC7
:100D4400022393FAA3F3B3FA83F303F01F0322FA03
:100D540003F313F0010FD9D029E0FFF747FB054651
:100D640007E0FFF743FB401B41F28833984200F24F
:100D74002A81022393FAA3F293FAA3F3B3FA83F337
:100D84005B0943F00203DBB2022B02D1394B1A6A2E
:100D940001E0384B5A6A022393FAA3F3B3FA83F3BC
:100DA40003F01F0322FA03F313F0010FD9D1E3690F
:100DB400022B04D940F24721304800F0BFFBE3691D
:100DC400002B00F002812B4A526802F00C02082A20
:100DD40000F0FD80022B40F0B780236A3BB1B3F5ED
:100DE400803F04D04FF41471244800F0A7FB636AD9
:100DF40073B3B3F5802F2BD0B3F5002F28D0B3F500
:100E0400402F25D0B3F5801F22D0B3F5A01F1FD0EB
:100E1400B3F5C01F1CD0B3F5E01F19D0B3F5001F04
:100E240016D0B3F5101F13D0B3F5201F10D0B3F5AF
:100E3400301F0DD0B3F5401F0AD0B3F5501F07D0B3
:100E4400B3F5601F04D040F251210C4800F076FB4A
:100E54004FF0807393FAA3F3B3FA83F39B0003F187
:100E6400844303F5840300221A60FFF7BFFA0546A2
:100E74000EE000BF0010024080044242E017000868
:100E840000700040FFF7B2FA401B022800F2A18074
:100E94004FF0007393FAA3F3514B1A684FF00073A9
:100EA40093FAA3F3B3FA83F303F01F0322FA03F3D1
:100EB40013F0010FE6D1236AB3F5803F10D1A36884
:100EC4003BB1B3F5003F04D040F26721454800F040
:100ED40035FB43494B6823F40032A36813434B604A
:100EE4003F48436823F47411236A626A13430B4333
:100EF40043604FF0807393FAA3F3B3FA83F39B0038
:100F040003F1844303F5840301221A60FFF76EFAA8
:100F1400044604E0FFF76AFA001B02285BD84FF08E
:100F2400007393FAA3F32E4B1A684FF0007393FAED
:100F3400A3F3B3FA83F303F01F0322FA03F313F0CA
:100F4400010FE7D0002049E04FF0807393FAA3F338
:100F5400B3FA83F39B0003F1844303F58403002273
:100F64001A60FFF743FA044604E0FFF73FFA001B58
:100F7400022832D84FF0007393FAA3F3184B1A687F
:100F84004FF0007393FAA3F3B3FA83F303F01F0350
:100F940022FA03F313F0010FE7D100201EE0012031
:100FA4001CE003201AE0032018E0012016E00320CF
:100FB40014E0032012E0032010E003200EE00320DD
:100FC4000CE003200AE0032008E0002006E00120F2
:100FD40004E0032002E0032000E0032003B030BD5E
:100FE40000100240E017000830B486B01F4D02AC78
:100FF40028686968AA68EB680FC42B8AADF80430C6
:101004001B4B5B6803F00C02082A2AD103F470110D
:101014004FF4701292FAA2F2B2FA82F221FA02F2B8
:1010240006A90A4412F8102C13F4803F15D0104B73
:101034005B6803F400314FF4003393FAA3F3B3FA7B
:1010440083F321FA03F306A90B4413F8140C094B98
:10105400B3FBF0F000FB02F004E0074800FB02F0F1
:1010640000E0044806B030BC704700BFCC1700084D
:101074000010024000127A0000093D0070B50D46D0
:10108400044620B94FF42F71A04800F057FA2368A2
:1010940013F00F0F04D140F2BD219C4800F04EFA2A
:1010A400022D04D940F2BE21984800F047FA984B2B
:1010B4001B6803F007039D420BD9954A136823F07C
:1010C40007032B431360136803F007039D4240F0AA
:1010D4000D81236813F0020F1DD0A368A3B1802BE8
:1010E40012D0902B10D0A02B0ED0B02B0CD0C02B34
:1010F4000AD0D02B08D0E02B06D0F02B04D040F23D
:10110400D721824800F01AFA82494B6823F0F00292
:10111400A36813434B60236813F0010F00F0818030
:101124006368022B04D940F2DE21784800F006FA05
:101134006268012A13D14FF4003393FAA3F3754B79
:1011440019684FF4003393FAA3F3B3FA83F303F06B
:101154001F0321FA03F313F0010F28D1C8E0022A78
:1011640013D14FF0007393FAA3F36A4B19684FF04D
:10117400007393FAA3F3B3FA83F303F01F0321FA82
:1011840003F313F0010F12D1B4E0022393FAA3F393
:10119400604B1968022393FAA3F3B3FA83F303F0C1
:1011A4001F0321FA03F313F0010F00F0A58059493E
:1011B4004B6823F0030313434B60FFF717F906460C
:1011C4006368012B0FD107E0FFF710F9801B41F290
:1011D4008833984200F292804E4B5B6803F00C0314
:1011E400042BF1D11DE0022B16D107E0FFF7FEF826
:1011F400801B41F28833984200F28280454B5B6841
:1012040003F00C03082BF1D10BE0FFF7EFF8801B80
:1012140041F28833984275D83E4B5B6813F00C0F4B
:10122400F3D13B4B1B6803F007039D420AD2384AB3
:10123400136823F007032B431360136803F00703B9
:101244009D4261D1236813F0040F19D0E36883B180
:10125400B3F5806F0DD0B3F5A06F0AD0B3F5C06FAE
:1012640007D0B3F5E06F04D040F23231274800F0E4
:1012740065F928494B6823F4E062E36813434B6043
:10128400236813F0080F1AD0236983B1B3F5806F74
:101294000DD0B3F5A06F0AD0B3F5C06F07D0B3F586
:1012A400E06F04D040F23931184800F047F9194A88
:1012B400536823F46053216943EAC1035360FFF781
:1012C40093FE144B5B6803F0F002F02393FAA3F34C
:1012D400B3FA83F322FA03F30F4AD35CD8400F4BDB
:1012E40018600020FFF754F8002070BD012070BD85
:1012F400012070BD012070BD012070BD032070BDB0
:10130400032070BD032070BD012070BDE0170008EC
:1013140000200240001002400C1800080C000020BD
:10132400014B1868704700BF0C000020FEE700BFA7
:1013340001230360014B0B60704700BF04000020D1
:1013440008B500F00FF8024B024A9A6008BD00BFCE
:1013540000ED00E00000000808B500F029F808BD21
:10136400FEE700000F4B1A6842F001021A60596848
:101374000D4A0A405A601A6822F0847222F48032BC
:101384001A601A6822F480221A605A6822F4FE0253
:101394005A604FF41F029A604FF00062034B9A6048
:1013A400704700BF001002400000FFF800ED00E0AD
:1013B4001F4B5B6803F00C03042B06D0082B08D0EA
:1013C4003BBB1C4A1C4B1A6026E01A4A1A4B1A6093
:1013D40022E0174A53685268C3F38343023312F47A
:1013E400803F05D1154A02FB03F3134A136013E04F
:1013F4000F4A526812F4003F05D0104A02FB03F36F
:101404000D4A136008E00B4A02FB03F30A4A136017
:1014140002E0084A084B1A60054B5B68C3F30313E8
:10142400074AD15C044A1368CB401360704700BF7D
:101434000010024000127A000C00002000093D0058
:101444000C18000810B586B0134B9A6942F01002CC
:101454009A619A6902F010020092009A9A6942F025
:1014640004029A619B6903F004030193019B0B4CF2
:1014740000224FF400512046FFF7FEF94FF40053C9
:101484000293012303930223059302A92046FFF745
:1014940057F806B010BD00BF001002400010014014
:1014A40008B500F0CDF8FEE700B591B0012306932E
:1014B4004FF4803307930022089202220D920E9378
:1014C4004FF4E0130F9306A8FFF700FA08B1FFF7F3
:1014D400E7FF0F23019302210291002303934FF4AA
:1014E40080620492059301A8FFF7C8FD08B1FFF7D5
:1014F400D7FFFFF715FF094BA3FB00308009FEF768
:10150400E9FF0420FEF7FCFF002211464FF0FF30F4
:10151400FEF79EFF11B05DF804FB00BFD34D6210CF
:1015240008B500F081F8FEF747FFFFF7BDFFFFF7AE
:1015340089FF00F087F800F07BF8FCE7704700BFF4
:1015440000B583B0204B9A6942F001029A619B690D
:1015540003F001030193019B0320FEF75BFF0022CC
:1015640011466FF00B00FEF773FF002211466FF077
:101574000A00FEF76DFF002211466FF00900FEF726
:1015840067FF002211466FF00400FEF761FF00229E
:1015940011466FF00300FEF75BFF002211466FF067
:1015A4000100FEF755FF002211464FF0FF30FEF711
:1015B4004FFF064A536823F0E06343F0007353601F
:1015C40003B05DF804FB00BF0010024000000140BE
:1015D400704700BFFEE700BFFEE700BFFEE700BFA5
:1015E400FEE700BF704700BF704700BF704700BFF1
:1015F40008B5FEF7F3FEFEF79FFF08BD08B54FF4EC
:1016040000510248FFF752F908BD00BF0010014025
:1016140008B54FF47A7300221146024800F02EF800
:1016240008BD00BF0116000808B500F00FF808BD9A
:1016340008B500F043F808BD08B500F06BF808BD24
:10164400704700BF08B5FFF7E3FF08BD30B40023BF
:101654000EE0094C9900CA189500601900226251E5
:1016640042600272C2602846204402610133DBB248
:101674000F2BEED930BC704720000020F0B50024B9
:1016840017E0274604EB8406B5000B4E3544ED689D
:101694006DB934464FEA870E0EEB0705AE00A51967
:1016A400A2516B6000232B72E8602961F0BD013404
:1016B400E4B20F2CE5D9F0BD2000002070B5002461
:1016C40022E004EB84029300114A1344DB68CBB19B
:1016D40004EB840293000E4A13441B7A93B1A100D5
:1016E40021448A000A4E1644013B3372F368306980
:1016F4009847736833B904EB8405AB00044A134478
:101704000022DA600134E4B20F2CDAD970BD00BFD4
:101714002000002070B400231FE003EB830082004C
:1017240010480244D268B2B103EB830082000D4832
:10173400825852B904469A00D518A80025186E6834
:101744002650287A411C297205E003EB83018800A6
:10175400013A04490A500133DBB20F2BDDD970BCC6
:10176400704700BF200000202E2E2F7379737465FC
:101774006D2F7372632F73746D3332663178782FE3
:1017840073746D3332663178785F68616C5F636F50
:10179400727465782E6300002E2E2F73797374652E
:1017A4006D2F7372632F73746D3332663178782FB3
:1017B40073746D3332663178785F68616C5F67701B
:1017C400696F2E6300000000020304050607080980
:1017D4000A0B0C0D0E0F1010010200002E2E2F7399
:1017E400797374656D2F7372632F73746D333266FE
:1017F4003178782F73746D3332663178785F68612D
:101804006C5F7263632E6300000000000000000040
:081814000102030406070809A4
:10181C00785634121C0000200000000000A24A047C
:04182C003254769824
:04000005080001E509
:00000001FF
